:100000000000000000000528090007309F0083164B
:100010009F01EB3086008A0183126E2882008207DE
:10002000063443346F346D346D346F346E3482076C
:10003000043444346F346E346534820704344634F7
:10004000613469346C3482070B344234493452349D
:100050004F34443432345F3454346534733474343C
:100060008207053449346E34703475347434820731
:10007000093449346E3474346534723472347534EE
:10008000703474348207143445346E34613462340D
:100090006C346534203461346E346434203441343B
:1000A0006C347434653472346E3461347434653451
:1000B000820704345234653461346434820708346E
:1000C000523465346734693473347434653472344B
:1000D000820704345434653473347434082424306F
:1000E000E300A8240824A60106161A245308A40035
:1000F000BB24BB2430302402031C8E283A30240257
:1001000003188E282408E200A224260DA700A70DBC
:10011000270DF8392407D03EA600FD2873302402AD
:10012000031D9B282408E200A22408242608D800E6
:100130004824A601FD2877302402031DC72824087F
:10014000E200A22408242608D8004824A601A5011C
:10015000033025020318B72842245708A70021308E
:1001600025078400270883138000A50AA828A50175
:10017000033025020318C528213025078400831386
:100180000008D5002924A50AB8280824FD286930CC
:100190002402031DD8282408E200A2240824FD30EC
:1001A000D80048247B237B237B2385238523FD28BC
:1001B00074302402031DE2282408E200A22408244B
:1001C0008D21FD2863302402031DEE282408E2005F
:1001D000A22408242608A800FE20FC283C30E200C7
:1001E000A2242408D50029243E30E200A2240824B9
:1001F0002608D50029240824A60174283B30B00025
:1002000028083002AF000230AA00FF30AB00F03007
:10021000AC005430E200A2240530D50029242F0878
:10022000D500292408244330E200A224FA30D80063
:10023000482442245708D5002924FB30D8004824FC
:10024000AE01AD01861A22292529861A2B29AE0A6C
:100250000319AD0A25294830E200A2242D08D50053
:1002600029244C30E200A2242E08D500292406308F
:100270002D020318602905302D02031C5B292E086E
:100280002F02031C53292F082E02031C4B29A901FE
:10029000AB01AC015229F830A9002F08B0002E089C
:1002A0003002AB005A29F930A9002E08B0002F08FF
:1002B0003002AB005F29F830A9002F08AB00672996
:1002C000F930A900FF30B0002F083002AB004530F4
:1002D000E200A2242B08D50029244D30E200A224FC
:1002E0002C08D50029242B082C02031D7A29082468
:1002F000003488292C082B02031C8529AA03031D1E
:100300008429AC0A0230AA0088292B08AC00AB0A69
:100310002908D800482408241329FA2297235F309B
:10032000E300A8246930E300A82408241030C300A7
:100330000330C4003030C500DA222030C30004305E
:10034000C4003130C500DA223030C3000530C400AB
:100350003230C500DA22B101E2210130B100E221E0
:100360000230B100E2210330B100E2213830E30075
:10037000A8246930E300A8240824BF010130C0008C
:100380002030C1000430C200BC220130BF00C001D7
:100390002030C1000130C200BC22BF010130C000CA
:1003A0003030C1000430C200BC220130BF00C001A7
:1003B0003030C1000130C200BC221830E300A82454
:1003C000082400343108BB0085220830B40034030F
:1003D000B50003303505B700370DBA003A0DFC39CA
:1003E0001038B600D800482437083105B800350C5D
:1003F000B900390C3F39B90006303904D800482417
:100400003508D50029243808D50029244330E300D5
:10041000A8246930E300A82408243230B2001E303A
:10042000B300BB24B30B112AB20B0F2A0330D80040
:10043000482442245708A0000F3036052002031933
:10044000292A2008D50029245930D1004030D20073
:100450000F240230D800482442245708A000390253
:100460000319372A5930D1004130D2000F24D80166
:10047000482442245708A00038020319472A2008BC
:10048000D50029245930D1004230D2000F24013048
:10049000D800482442245708A00038020319582ADB
:1004A0002008D50029245930D1004330D2000F2430
:1004B00003303604D8004824D80148244224570881
:1004C000A00003302006380203196E2A2008D50048
:1004D00029245930D1004430D2000F240130D800F3
:1004E000482442245708A000380203197F2A200814
:1004F000D50029245930D1004530D2000F243608C8
:10050000D8004824B40BE72900341C30D800482414
:1005100008243B0AA00020083B020319AB2A0D3037
:10052000E200A2243130E300A8243B08BD00AD2244
:100530003C30E200A2242008BD00AD223E30E200A3
:10054000A2243A30E200A2240130D80048244224F8
:100550005708A0008B2A08240034BD183130BD1C78
:100560003030BE00E200A2243D1831303D1C303056
:10057000BE00E200A22400343F08BB0085221430F4
:10058000D800482441084204D80048244008BD004F
:10059000AD223A30E200A224D1224108D8004824FA
:1005A0000034F230D8004824861ED82ABB24D42A2E
:1005B000082400341030C60046080319F92AC6037F
:1005C00043084604D80048244408D800482442245C
:1005D0005708A00046020319F82A4608D500292426
:1005E0002008D50029245F30D1004508D2000F240F
:1005F000DC2A0034FD30D80048240130C900C03066
:10060000CA007023C901C130CA0070230B30C90071
:10061000C230CA0070230130C900C330CA00702341
:10062000C901C430CA007023C901C530CA00702393
:10063000C901C630CA007023C901C730CA0070237F
:1006400008247B237B238523852390234D08FD30BD
:10065000D80048240130C900C830CA007023FE30D9
:10066000D800482442245708C700FF30D800482447
:10067000FF30D8004824FE30D800482442245708D0
:10068000C8000230480203194A2B1030D100C9308B
:10069000D2000F24FB30D800482442245708031905
:1006A000562B1030D100CA30D2000F24FA30D800B7
:1006B000482442245708C700F930D8004824F830AD
:1006C000D8004824FA30D80048244224570847026A
:1006D00003196F2B1030D100CB30D2000F2400341F
:1006E00090234D08490203197A2B1030D1004A0893
:1006F000D2000F2400340830CB0090234D08D500E1
:100700002924CB0B7D2B0824003490234D08CC00EA
:1007100090234D08E200A224CC0B882B082400343F
:10072000FC30D800482442245708CD000034F03073
:10073000D8004824CF01D030D000F623F530D800BF
:1007400048240130CF00D130D000F623F430D80057
:100750004824CF01D230D000F623F130D80048240D
:100760000130CF00D330D000F623F030D800482439
:10077000CF01D430D000F623F730D800482402301F
:10078000CF00D530D000F623F630D8004824CF0172
:10079000D630D000F623F230D80048240230CF0003
:1007A000D730D000F623F030D8004824CF01D8301D
:1007B000D000F623F330D80048240330CE00BB2409
:1007C000CE0BDF2B861EE92B3830D100D930D2007A
:1007D0000F240130CF00DA30D000F623F030D800FB
:1007E0004824CF01DB30D000F6230034EF30D800AE
:1007F000482442245708A0004F020319072C200860
:10080000D50029243830D1005008D2000F240034FC
:100810000D30E200A2240A30E200A22400341E308F
:10082000E300A8245108E300A8245208D500292495
:1008300008240034FC30D400FC305402031D262C64
:100840000230D9004E245A08D4001C2C5408D3007E
:100850000034550ED600D60C560C0339303EE2005B
:10086000A224550CD600D60C560C0739303EE200B7
:10087000A22407305505303EE200A2242030E200D9
:10088000A22400342030D9004E245A08D700003466
:100890005808DE001030DF007C240034DB0106083D
:1008A000590503195C2CDB035B08031D5A2CFC3033
:1008B000DA000034BB244F2CBB24BB24BB24DC0156
:1008C0000230DD00DD0B622C000000000830DB0090
:1008D000BB240310DC0C06085905031DDC17BB24E0
:1008E000BB240000000000000000DB0B682CBB24D0
:1008F000BB245C08DA000034FF305F06E1008600AC
:10090000BB24BB24BB24000000000000000000004A
:1009100000000830E0005E18FF305E1C61088600B1
:100920000310DE0CBB24BB24BB2400000000E00B42
:100930008B2C0000FF308600BB24BB24BB240000AE
:10094000000000346208DE000430DF007C24003444
:10095000E5018A0163080E2065020318B72C650AB9
:1009600063078A010E20E200A224E50AA92C2030A8
:10097000E200A224003464007030E600E60BBE2CD6
:04098000000000343F
:02400E00293F48
:00000001FF
